:020000040000FA
:10000000AF01A501F00113280308F2008B1E0D2893
:100010000B11F00A72088300090083120C10F10A18
:10002000720883000900FF30850086016400831692
:1000300004308100E03085007A3086008312303051
:1000400090000130AB000230B000B300830180307B
:100050008B0006087039703CF3000310F30CF30CAE
:10006000F30CF30C402083160313990024309800FE
:1000700005307302031818118301903098004D2841
:1000800000308A007308031082070A3415342034C4
:1000900040348134413441344134AD230130AD002A
:1000A0000511D2200515EE20A301A5014E28003030
:1000B0008A0003102B0D8207212561282C25612839
:1000C0003A252808A0009620A90B57280800782078
:1000D0002008A70000308A0003102B0D820751254D
:1000E00074287C2574289625A90B6728A30108008D
:1000F0003408A000A3033508B4003608B50037085B
:10010000B6003808B70008003908A000A5033A086F
:10011000B9003B08BA0008003308A000FE30810097
:100120000B110B1D9128A00B8E28080000308A00AF
:100130000310250DA400A40D240882072008B9008F
:100140000000A9282008BA000000A9282008BB0048
:100150000000A50A080000308A000310230DA40047
:10016000A40D240882072008B4000000C528200838
:10017000B5000000C5282008B6000000C5282008EA
:10018000B7000000C5282008B800A30A08000C1E0C
:10019000C728A50803190800842020089900AC0B83
:1001A000C7280800861DD6280614D22806108C1AE7
:1001B000DC28861DD728D22818080239031DE62816
:1001C0001A08A000AB20AD0BD7280800181218168B
:1001D0000030A000AB20AD0BE8280800A3080319ED
:1001E0000800E03034020319DC2AE8303402031935
:1001F000DC2AC03034020319EF2AC8303402031954
:10020000EF2A0E30340203193A2A0C303402031953
:10021000682A423034020319C02A623034020319BA
:10022000992A053034020319B32A703034020319B5
:100230008A2A773034020319FC2AE4303402031985
:10024000DC2AEC3034020319DC2AC43034020319EE
:10025000EF2ACC3034020319EF2A63303402031939
:10026000992A643034020319992A6530340203193B
:10027000992A663034020319992A67303402031927
:10028000992A6830340203198A2A69303402031922
:100290008A2A6B3034020319992A6F303402031909
:1002A000992A6C3034020319992A43303402031915
:1002B000C02A443034020319C02A453034020319DD
:1002C000C02A463034020319C02A473034020319C9
:1002D000C02A843034020319B32A9430340203193B
:1002E000B32A4B3034020319C02A4C3034020319AC
:1002F000C02A2D30340203191E2D90303402031908
:100300001E2A083034020319192A10303402031946
:100310001E2A183034020319192AD5303402031961
:10032000052AD63034020319132AE53034020319A2
:10033000272AC53034020319322A8E3034020319B9
:100340007F2AE130340203194E2AC13034020319E6
:100350000F2D2E30340203195D2AE23034020319C6
:10036000762A713034020319A82A15303402031991
:10037000CD2A543034020319412B52303402031970
:10038000AD2B4D3034020319EF2C503034020319D9
:10039000F72C763034020319012DFA303402031998
:1003A000D22BDF3034020319D22BBF3034020319B1
:1003B000D22BBE3034020319D22BFE303402031983
:1003C000082D573034020319F62956303402031928
:1003D000F929533034020319FC295530340203192A
:1003E000FF29513034020319022A08002030C200CC
:1003F000422C0530C200422C4030C200422C413019
:10040000C200422C6030C200422C0130C000A90062
:10041000C1006720FF3A0319C001A00096200130F7
:10042000AC00C72008000130A90067208C20C00163
:1004300008000130A90067208C2008000130A900C5
:100440004008C1006720C00803198C200800341040
:100450000130A90067200130A90057200130AC000D
:10046000C720080034100130AD00D2200230A900AE
:1004700067200800B40E0230AD00D220061403300D
:10048000A9004008C1006720C00803198C20013072
:10049000A90057200130AC00C72008000230AD0091
:1004A000D22006140330A90067208C200230A90056
:1004B00057200230AC00C7200800B40E0130A9005C
:1004C00067200230A90057200230AC00C720080086
:1004D000B40E0330AD00D22006140430A900400849
:1004E000C1006720C00803198C200800B412023034
:1004F000AD00D22006140330A90067200800B40E16
:100500000130A90067200230A90057200230AC005A
:10051000C72008000130A9004008C1006720C008BA
:1005200003198C200130A90057200130AC00C720EE
:1005300008000130A9004008C1006720C008031965
:100540008C200230A90057200230AC00C7200800E0
:100550000130A90067208C200230A900572002300A
:10056000AC00C7200800B40E0130AD00D22002302C
:10057000A9004008C1006720C00803198C200800AA
:100580000230AD00D22006140330A9004008C1009B
:100590006720C00803198C200800B40E0130AD009C
:1005A000D2200230A90067208C200130A9005720FA
:1005B0000130AC00C72008000230AD00D220061484
:1005C0000330A9004008C1006720C00803198C202F
:1005D0000230A90057200230AC00C72008000430C8
:1005E000AD00D22006140530A9004008C1006720E4
:1005F000C00803198C2008000614A301051281010C
:100600000B110B1D012B05160B118B16051E0B2B49
:10061000F01B332B062BF001B101051A142BF01B34
:10062000332B0000B10A0D2B8B12310AB000B2003F
:100630000310B00C0310B00C3008B30003303002CC
:100640000318262BB0033008AB00312B0230AB006F
:100650003008B100B0010330B00AB10203182B2BEF
:10066000B0033208392B0130AB000230B000B300C8
:100670000301A0008B1296200130AC00C720F001CE
:100680000800A3010130AD00D22003308A0003101E
:10069000340DA400A40D240D82070730B0002130D2
:1006A000B3000230AB00000008000430B00014308A
:1006B000B3000230AB00000008000330B00010307F
:1006C000B3000230AB00000008000230B000083078
:1006D000B3000230AB00000008000230B000073069
:1006E000B3000230AB00000008000230B00006305A
:1006F000B3000230AB00000008000130B00005304C
:10070000B3000230AB00000008000130B00004303C
:10071000B3000230AB00000008000130B00003302D
:10072000B3000230AB00000008000230B00002301D
:10073000B3000130AB00000008000230B00002300E
:10074000B3000130AB00000008000130B000013000
:10075000B3000030AB0000000800A301C001061484
:10076000AF1C8514AF1885102F1C05142F18051009
:100770002F1D05122F19051686170A30A00001300B
:1007800081000B110B1DC22BA00BBF2B8613033056
:10079000A000013081000B110B1DCC2BA00BC92B2D
:1007A00005160800B40985150330AD00D2200614E3
:1007B0003408C2003508C3003608C4003708C70033
:1007C0002030B6002724A501B91F402C4308B500EE
:1007D0004408B6004708B7001B241830B50026307F
:1007E000B6004208B7001B241830B5002530B6000B
:1007F0008030B7001B24F1018F018E010C10101402
:1008000083160C1483127119382C2530B600831608
:100810000C1083122724A501B91A132C391A132C92
:10082000391F002C3E2C1830B5002530B600303072
:10083000B7001B24002CC030B4000430A300A90072
:100840004008C1006720C00803198C200800E03070
:10085000B4001830B5000330A300A9004008C1005F
:100860006720C00803198C200130A9005720080018
:1008700083160C1083121010F230E62C0030E62C98
:10088000F130E62C8515A3010430AD00D22006140A
:100890003408C3003508C4003608C5003708C60050
:1008A000A301E030B40001304807B5004908B600A4
:1008B0000330A300BB24A501B91FE52CC830A0005C
:1008C000AB204308A000AB204408A000AB204508A3
:1008D000A000AB204608A000AB20B2240630A10047
:1008E0004208A200C7240530A1008030A200C7241E
:1008F000F1018F018E010C10101483160C14831259
:100900007119DD2CE030A000AB20A00105304907B3
:10091000A100A00D2008013E4807A000AB2021083F
:10092000A000AB2083160C108312BB24A501BA18BB
:10093000AC2CBA1AA62C3A1AA02C3A1F7D2CE32C08
:100940000530A1001030A200C7247D2C0530A10085
:100950002030A200C7247D2C0530A1000330A20066
:10096000C7247D2C0530A9004008C1006720C008BD
:1009700003198C2008000330A9004008C10067203B
:10098000C00803198C200230A90057200800C0308D
:10099000A000AB20A00121084907A100A00D20085C
:1009A000013E4807A000AB202108A000AB20220890
:1009B000A000AB20AB20B224080083160C108312D9
:1009C0001010F230E62C0030E62CF130B900A50111
:1009D000A301A50A0130AC00C72085110800A301BE
:1009E0000130AD00D22034080739AF000800A30160
:1009F0000230AD00D220A3013408C8003508C90078
:100A000008001530A00096200130AC00C720080077
:100A10000030A00096200130AC00C7200800033051
:100A2000AD00D22006140430A90067208C200130CC
:100A3000A90057200130AC00C72008004D30B40099
:100A4000C02A0830A600051205160310051A031463
:100A5000A80DA60B232D08000830A60005120000E3
:100A60000516000000000310051A0314A80DA60BBC
:100A70002E2D08000830A6003008BC00BD00BE00C6
:100A80000512BC0B412D0516BD0B442D0310BE0DE8
:100A9000051A0314A80D0000BE0B4B2DA60B3C2D10
:100AA00008000830A600A70D031C5C2D05120516D2
:100AB0000000A60B532D652D05120000000000005C
:100AC000000000000516A60B532D41082906031D42
:100AD000080081010B118B16051E722DF01B772D5E
:100AE000051A6C2D8B12051E732D0301792D8B12A7
:100AF000FF30F001C10108000830A6000330BD003E
:100B0000A70D031C8B2D842D051200000516000077
:100B1000A60B7E2D912D0512BD0B8C2D0516A60B57
:100B20007E2D41082906031D0800692D0830A60006
:100B30003008BF00BF07BF07BF07BF07BF073008A8
:100B4000BC003F08BD00A70D031CAF2D0512BC0B58
:100B5000A72D0516BD0BAA2DA60B9F2DB52D051291
:100B6000BD0BB02D0516A60B9F2D41082906031DB0
:040B70000800692DE3
:02400E00223F4F
:00000001FF
